:0200000480007A
:10000000373500FF13050530930570002322B50036
:1000100003264500130500006B000500938B0600C6
:10002000130D0700130F01009303050013051000C3
:10003000635C750013010180130305006B5003001E
:10004000130515006FF0DFFE130000001300000021
:100050001300000013000000130000001300000054
:1000600013010F0013050000930F0600938D03008A
:100070001300000013000000130000001300000034
:100080001300000013000000130000001300000024
:10009000EBE0BF011300000013000000130000009C
:1000A00013000000130000001300000017050000FB
:1000B0001305451B6B40050017030000130343F6AF
:1000C0006B00030067800000170200011302822406
:1000D00023200200232212002324220023263200A0
:1000E00023284200232A5200232C6200232E720070
:1000F00023208202232292022324A2022326B20278
:100100002328C202232AD202232CE202232EF20247
:10011000232002052322120523242205232632054B
:1001200023284205232A5205232C6205232E72051B
:1001300023208207232292072324A2072326B20723
:100140002328C207232AD207232CE207232EF207F3
:100150001302100067800000170200011302821BC7
:100160000320020083204200032182008321C20079
:100170000322020183224201032382018323C2015D
:100180000324020283244202032582028325C20241
:100190000326020383264203032782038327C20325
:1001A0000328020483284204032982048329C20409
:1001B000032A0205832A4205032B8205832BC205ED
:1001C000032C0206832C4206032D8206832DC206D1
:1001D000032E0207832E4207032F8207832FC207B5
:1001E0001302000067800000732500026780000092
:1001F0007325100267800000130101FE232E1100F9
:10020000232C810013040102232604FE6F00400307
:100210000327C4FEB7170000938747973307F702F9
:10022000B707008193870741B307F70013850700DD
:10023000EF0000448327C4FE938717002326F4FEB3
:100240000327C4FE9307F001E3D4E7FC130000008A
:100250008320C10103248101130101026780000092
:10026000130101FD23261102232481022322A1036D
:10027000130401031300000013070D00B71700005B
:10028000938747973307F702B707008193870741A2
:10029000B307F70013850700EF00405093070500F0
:1002A000638A070213070D00B707008113172700A1
:1002B00093878726B307F7001307100023A0E700F2
:1002C00093070D0063960700EFF01FE96F00C0056C
:1002D0007300000013070D00B717000093874797BE
:1002E0003307F702B707008193870741B307F70089
:1002F000130784FD9305070013850700EF000040F6
:10030000832704FE138107008327C4FD832584FD12
:10031000032644FE832684FE0327C4FE13850700BC
:10032000EFF0DFCF730000008320C10203248102BD
:10033000032D41021301010367800000130101FB3B
:10034000232611042324810413040105EFF0DFE9BF
:100350002324A4FE93090100930710002326F4FE32
:100360006F00C0080327C4FEB717000093874797A4
:100370003307F702B707008193870741B307F700F8
:1003800013850700EF00804193070500639A070477
:100390000327C4FEB7170000938747973307F70278
:1003A000B707008193870741B307F700130704FDE0
:1003B0009305070013850700EF004034832784FD71
:1003C00013810700832744FD832504FD0326C4FD14
:1003D000832604FE032744FE13850700EFF0DFCDDC
:1003E0008327C4FE938717002326F4FE8327C4FEC9
:1003F000032784FEE3E8E7F613810900EFF0DFCC82
:100400009307020063880704B7070081138507413B
:10041000EF00C03893070500639E0702930784FB33
:1004200093850700B707008113850741EF00002D72
:10043000832704FC138107008327C4FB832584FBE7
:10044000032644FC832684FC0327C4FC1385070091
:10045000EFF0DFBC130000008320C10403248104FB
:100460001301010567800000130101FB232611041D
:100470002324810413040105232EA4FA232CB4FAA7
:10048000232AC4FA2328D4FAEFF01FD7EFF0DFD5E0
:100490002322A4FE13090100232604FE232404FEC4
:1004A0006F000009B709FFFF33013101832784FE84
:1004B0002326F4FC832784FB2328F4FC9307010004
:1004C000232AF4FC832744FB232CF4FC832704FB1E
:1004D000232EF4FC8327C4FE2320F4FE0327C4FE4E
:1004E000B7170000938747973307F702B7070081D4
:1004F00093870741B307F7001307C4FC9305070070
:1005000013850700EF0000198327C4FE93871700A7
:100510002326F4FE8327C4FE032744FE63E4E7009A
:10052000232604FE832784FE938717002324F4FEEA
:10053000032784FE8327C4FBE366F7F61301090053
:10054000EFF0DFDF130000008320C10403248104E7
:100550001301010567800000130101FD232611022C
:100560002324810213040103232EA4FC8325C4FD4C
:10057000B707008113850704EF004035EFF0DFC6B1
:100580002320A4FE232604FE6F008006930710009C
:100590002326F4FE232404FE6F00C003B707008166
:1005A000032784FE1317270093878726B307F700D6
:1005B00003A70700930710006318F7008327C4FE02
:1005C000938717002326F4FE832784FE9387170062
:1005D0002324F4FE032784FE9307F001E3D0E7FC15
:1005E0008325C4FEB70700811385C704EF00002EE2
:1005F0000327C4FE8327C4FDE36AF7F8232204FE21
:100600006F008002B7070081032744FE13172700FD
:1006100093878726B307F70023A00700832744FEAC
:10062000938717002322F4FE832744FE032704FE4A
:10063000E3EAE7FC130000008320C10203248102E7
:100640001301010367800000130101FF23268100CD
:10065000232471011304010193870B001385070004
:100660000324C100832B8100130101016780000076
:1006700093020500130300009303700023A062009F
:1006800023A2620023A4620023A6720023A86200B2
:10069000678000009302050003A382001303130088
:1006A00023A462001383420183AE420093935E0051
:1006B0003303730003AE05002320C30103AE4500DE
:1006C0002322C30103AE85002324C30103AEC5006A
:1006D0002326C30103AE05012328C30103AE450150
:1006E000232AC301938E1E00130F20036394EE018F
:1006F000930E000023A2D201678000009302050040
:1007000003A3820013000000130000001300000088
:100710001300000013000000130000001303F3FF98
:1007200023A462001383420183AE0200930F2003CF
:10073000138F0E00130F1F006314FF01130F00002F
:1007400023A0E20193935E0033037300032E0300A2
:1007500023A0C501032E430023A2C501032E83005D
:1007600023A4C501032EC30023A6C501032E030144
:1007700023A8C501032E430123AAC50167800000F9
:100780009302050003A3820013050000130E20034B
:1007900063146E00130515006780000093020500C6
:1007A00003A3820013050000130E000063146E0003
:1007B00013051500678000009302050003A3C20023
:1007C00083A3020133B5630067800000130141FF7A
:1007D000232011002322B100834505006388050012
:1007E000EF00C001130515006FF01FFF832001000B
:1007F000832541001301C10067800000B708010094
:1008000023A0B80067800000130101FD2326110218
:100810002324810213040103232EA4FC0327C4FD17
:100820009307F00063E4E702B70700810327C4FDE4
:10083000131727009387871AB307F70083A70700CA
:1008400013850700EFF09FF86F0040079307000241
:100850002326F4FEA30504FE8327C4FE9387C7FF67
:100860000327C4FDB357F70093F7F7002322F4FEE4
:10087000832744FE6386070093071000A305F4FE58
:100880008347B4FE63820702B7070081032744FE53
:10089000131727009387871AB307F70083A707006A
:1008A00013850700EFF09FF28327C4FE9387C7FFED
:1008B0002326F4FE8327C4FEE340F0FA8320C1021E
:1008C000032481021301010367800000130101FE6C
:1008D000232E1100232C8100130401022326A4FEE1
:1008E0002324B4FE0325C4FEEFF05FEE032584FE4F
:1008F000EFF09FF1B707008113854709EFF01FED77
:10090000130000008320C1010324810113010102AF
:1009100067800000130101FD2326110223248102B8
:1009200013040103232EA4FC232CB4FC232AC4FCAF
:100930002328D4FCB76702810327C4FD23ACE71A40
:10094000B76702819387871B032784FD23A2E700F3
:10095000B76702819387871B032744FD23A4E70021
:10096000B76702819387871B032704FD23A6E7004F
:10097000EFF01F882324A4FE032704FD832784FEB1
:10098000B357F7022326F4FE032704FD832784FED2
:10099000B377F702638807008327C4FE93871700A5
:1009A0002326F4FEB76702819387871B0327C4FEC3
:1009B00023A8E700032704FD832784FE6362F70270
:1009C000B76702819386871BB7170080138687A3BA
:1009D000832584FE032504FDEFF01FA96F000002AC
:1009E000B76702819386871BB7170080138687A39A
:1009F000832504FD032504FDEFF01FA7EFF0CFFED4
:100A00002322A4FE032704FD832744FE63F8E700A6
:100A1000032544FEEFF05FB46F00C000032504FD22
:100A2000EFF09FB3130000008320C1020324810272
:100A30001301010367800000130101FA232E110442
:100A4000232C8104130401062326A4FA2324B4FAD8
:100A5000EFF09FBF232CA4FC832784FD83A707000E
:100A6000232AF4FC832784FD83A747002328F4FC72
:100A7000832784FD83A787002326F4FC832784FD36
:100A800083A707012326F4FE0327C4FE8327C4FAA5
:100A9000B307F7022324F4FE8327C4FE639A0700FA
:100AA000930710002326F4FE8327C4FA2324F4FEC0
:100AB000832784FD83A7C7002324F4FC232204FE9C
:100AC0006F00800D232004FE232E04FC6F0080079E
:100AD000032784FA832784FCB307F7020327C4FDA6
:100AE000B307F7002322F4FC032784FC8327C4FD0B
:100AF000B307F702032784FEB307F7002320F4FCB3
:100B0000832744FC93972700032744FDB307F7008E
:100B100003A70700832704FC93972700832604FD7F
:100B2000B387F60083A70700B307F702032704FE85
:100B3000B307F7002320F4FE8327C4FD9387170033
:100B4000232EF4FC0327C4FD832784FCE362F7F81B
:100B5000032784FA832784FC3307F702832784FE64
:100B6000B307F700232EF4FA8327C4FB93972700DB
:100B70000327C4FCB307F700032704FE23A0E70004
:100B8000832784FE938717002324F4FE832744FEE3
:100B9000938717002322F4FE832744FE0327C4FE15
:100BA000E3E2E7F2130000008320C105032481057E
:100BB0001301010667800000130101FC232E1102BE
:100BC000232C810213040104232EA4FC232CB4FC47
:100BD000232AC4FC2328D4FC2326E4FCB767028123
:100BE0000327C4FD23A6E71CB76702819387C71CB0
:100BF000032784FD23A2E700B76702819387C71C00
:100C0000032744FD23A4E700B76702819387C71C2D
:100C10000327C4FC23A6E700B76702819387C71C9C
:100C2000032704FD23A8E700EFF08FDC2324A4FEB4
:100C30000327C4FC832784FEB357F7022326F4FE60
:100C40000327C4FC832784FEB377F7026388070079
:100C50008327C4FE938717002326F4FEB76702811B
:100C60009387C71C0327C4FE23AAE7000327C4FCFD
:100C7000832784FE6362F702B76702819386C71CED
:100C8000B7170080138607CF832584FE032504FD54
:100C9000EFF08FFD6F000002B76702819386C71CDB
:100CA000B7170080138607CF8325C4FC032504FDF6
:100CB000EFF08FFBEFF04FD32322A4FE032704FDB8
:100CC000832744FE63F8E700032544FEEFF0DF8846
:100CD0006F00C000032504FDEFF01F881300000023
:100CE0008320C103032481031301010467800000F2
:100CF000130101FB2326110423248104130401059D
:100D0000232EA4FA232CB4FAEFF01F942320A4FE80
:100D1000832704FE83A70700232EF4FC832704FE09
:100D200083A74700232CF4FC832704FE83A78700B6
:100D3000232AF4FC832704FE83A747012326F4FE1D
:100D40000327C4FE8327C4FBB307F7022324F4FE62
:100D50008327C4FE639A0700930710002326F4FE3E
:100D60008327C4FB2324F4FE832704FE83A7C70044
:100D70002328F4FC232204FE6F00000C032784FBCD
:100D8000832704FD3307F702832784FEB307F700A8
:100D90002326F4FC032784FE832704FDB337F700E2
:100DA00093F7F70F2324F4FC832784FC93B71700F1
:100DB000A303F4FC834774FC138F0700B71700806C
:100DC000938F47E26B200F007B70FF018327C4FCE9
:100DD000939727000327C4FDB307F70083A60700F6
:100DE0008327C4FC93972700032784FDB307F700EC
:100DF00003A707008327C4FC93972700032644FD1D
:100E0000B307F6003387E60023A0E700832784FEBC
:100E1000938717002324F4FEB7170080138E87E210
:100E200067000E00130000006B300000832744FEB3
:100E3000938717002322F4FE832744FE0327C4FE72
:100E4000E3EEE7F2130000008320C10403248104D1
:100E50001301010567800000130101FC232E11021C
:100E6000232C810213040104232EA4FC232CB4FCA4
:100E7000232AC4FC2328D4FC2326E4FCB767028180
:100E80000327C4FD23A6E71CB76702819387C71C0D
:100E9000032784FD23A2E700B76702819387C71C5D
:100EA000032744FD23A4E700B76702819387C71C8B
:100EB0000327C4FC23A6E700B76702819387C71CFA
:100EC000032704FD23A8E700EFF08FB22324A4FE3C
:100ED0000327C4FC832784FEB357F7022326F4FEBE
:100EE0000327C4FC832784FEB377F70263880700D7
:100EF0008327C4FE938717002326F4FEB767028179
:100F00009387C71C0327C4FE23AAE7000327C4FC5A
:100F1000832784FE6362F702B76702819386C71C4A
:100F2000B7170080138607F9832584FE032504FD87
:100F3000EFF08FD36F000002B76702819386C71C62
:100F4000B7170080138607F98325C4FC032504FD29
:100F5000EFF08FD1EFF04FA92322A4FE032704FD69
:100F6000832744FE63F8E700032544FEEFF0CFDE5D
:100F70006F00C000032504FDEFF00FDE130000003A
:100F80008320C1030324810313010104678000004F
:100F9000130101FB232611042324810413040105FA
:100FA000232EA4FA232CB4FAEFF00FEA2320A4FE98
:100FB000832704FE83A70700232EF4FC832704FE67
:100FC00083A74700232CF4FC832704FE83A7870014
:100FD000232AF4FC832704FE83A747012326F4FE7B
:100FE0000327C4FE8327C4FBB307F7022324F4FEC0
:100FF0008327C4FE639A0700930710002326F4FE9C
:101000008327C4FB2324F4FE832704FE83A7C700A1
:101010002328F4FC232204FE6F00000C032784FB2A
:10102000832704FD3307F702832784FEB307F70005
:101030002326F4FC032784FE832704FDB337F7003F
:1010400093F7F70F2324F4FC832784FC93B717004E
:10105000A303F4FC834774FC138F0700B7170080C9
:10106000938F470C6B200F007B70FF018327C4FC1C
:10107000939727000327C4FDB307F70083A6070053
:101080008327C4FC93972700032784FDB307F70049
:1010900003A707008327C4FC93972700032644FD7A
:1010A000B307F6003387E64023A0E700832784FEDA
:1010B000938717002324F4FEB7170080138E870C44
:1010C00067000E00130000006B300000832744FE11
:1010D000938717002322F4FE832744FE0327C4FED0
:1010E000E3EEE7F2130000008320C104032481042F
:1010F0001301010567800000130101FC232E11027A
:10110000232C810213040104232EA4FC232CB4FC01
:10111000232AC4FC2328D4FC2326E4FCB7670281DD
:101120000327C4FD23A2E71EB76702819387471EEA
:10113000032784FD23A2E700B76702819387471E38
:10114000032744FD23A4E700B76702819387471E66
:101150000327C4FC23A6E700B76702819387471ED5
:10116000032704FD23A8E700EFF08F882324A4FEC3
:101170000327C4FC832784FEB357F7022326F4FE1B
:101180000327C4FC832784FEB377F7026388070034
:101190008327C4FE938717002326F4FEB7670281D6
:1011A0009387471E0327C4FE23AAE7000327C4FC36
:1011B000832784FE6362F702B76702819386471E26
:1011C000B717008013860723832584FE032504FDBB
:1011D000EFF08FA96F000002B76702819386471E68
:1011E000B7170080138607238325C4FC032504FD5D
:1011F000EFF08FA7EFE05FFF2322A4FE032704FD9B
:10120000832744FE63F8E700032544FEEFF0CFB4E4
:101210006F00C000032504FDEFF00FB413000000C1
:101220008320C103032481031301010467800000AC
:10123000130101FB23261104232481041304010557
:10124000232EA4FA232CB4FAEFF00FC02320A4FE1F
:10125000832704FE83A70700232EF4FC832704FEC4
:1012600083A7470083A70700232CF4FC832704FEF1
:1012700083A78700232AF4FC832704FE83A7470162
:101280002326F4FE0327C4FE8327C4FBB307F7021B
:101290002324F4FE8327C4FE639A070093071000FB
:1012A0002326F4FE8327C4FB2324F4FE832704FEB5
:1012B00083A7C7002328F4FC232204FE6F00000B41
:1012C000032784FB832704FD3307F702832784FE6B
:1012D000B307F7002326F4FC032784FE832704FDCD
:1012E000B337F70093F7F70F2324F4FC832784FC2C
:1012F00093B71700A303F4FC834774FC138F070014
:10130000B7170080938F87356B200F007B70FF012C
:101310008327C4FC939727000327C4FDB307F70076
:1013200083A607008327C4FC93972700032744FD67
:10133000B307F700032784FD3387E60023A0E70007
:10134000832784FE938717002324F4FEB7170080B9
:10135000138EC73567000E00130000006B300000CD
:10136000832744FE938717002322F4FE832744FE3D
:101370000327C4FEE3E6E7F4130000008320C10462
:10138000032481041301010567800000130101FC9F
:10139000232E1102232C810213040104232EA4FC0A
:1013A000232CB4FC232AC4FC2328D4FC2326E4FCED
:1013B000B76702810327C4FD23A2E71EB767028136
:1013C0009387471E032784FD23A2E700B7670281A6
:1013D0009387471E032744FD23A4E700B7670281D4
:1013E0009387471E0327C4FC23A6E700B767028143
:1013F0009387471E032704FD23A8E700EFE05FDF84
:101400002324A4FE0327C4FC832784FEB357F702DA
:101410002326F4FE0327C4FC832784FEB377F70258
:10142000638807008327C4FE938717002326F4FEF2
:10143000B76702819387471E0327C4FE23AAE700EC
:101440000327C4FC832784FE6362F702B767028127
:101450009386471EB71700801386474C832584FE6A
:10146000032504FDEFF04F806F000002B767028193
:101470009386471EB71700801386474C8325C4FC0C
:10148000032504FDEFE05FFEEFE01FD62322A4FE5C
:10149000032704FD832744FE63F8E700032544FE89
:1014A000EFF08F8B6F00C000032504FDEFF0CF8AB3
:1014B000130000008320C1030324810313010104EE
:1014C00067800000130101FB2326110423248104FB
:1014D00013040105232EA4FA232CB4FAEFF0CF96BF
:1014E0002320A4FE832704FE83A70700232EF4FCF9
:1014F000832704FE83A7470083A70700232CF4FC5F
:10150000832704FE83A78700232AF4FC832704FE95
:1015100083A747012326F4FE0327C4FE8327C4FBC9
:10152000B307F7022324F4FE8327C4FE639A07005F
:10153000930710002326F4FE8327C4FB2324F4FE24
:10154000832704FE83A7C7002328F4FC232204FE7C
:101550006F00000B032784FB832704FD3307F7028A
:10156000832784FEB307F7002326F4FC032784FEB9
:10157000832704FDB337F70093F7F70F2324F4FC18
:10158000832784FC93B71700A303F4FC834774FC00
:10159000138F0700B7170080938FC75E6B200F0073
:1015A0007B70FF018327C4FC939727000327C4FDAA
:1015B000B307F70083A607008327C4FC939727008F
:1015C000032744FDB307F700032784FD3387E602B2
:1015D00023A0E700832784FE938717002324F4FECB
:1015E000B7170080138E075F67000E00130000001E
:1015F0006B300000832744FE938717002322F4FEFC
:10160000832744FE0327C4FEE3E6E7F4130000004B
:101610008320C104032481041301010567800000B5
:10162000130101FD2326810213040103232EA4FCD0
:10163000232604FE6F0000018327C4FE9387170052
:101640002326F4FE0327C4FE8327C4FDE346F7FEEA
:10165000130000000324C10213010103678000008E
:10166000130101FD23261102232481021304010327
:10167000232EA4FC232CB4FCB76702811387C71F59
:101680008327C4FDB307F700130710002380E7008A
:101690008327C4FD6390070CA30104FE232604FEE8
:1016A0006F00800A232604FE232404FE6F004003FB
:1016B000B76702811387C71F832784FEB307F7002C
:1016C00083C70700638807008327C4FE938717003A
:1016D0002326F4FE832784FE938717002324F4FE39
:1016E000032784FE832784FDE344F7FC0327C4FE1D
:1016F000832784FD631AF704232204FE6F0000048D
:10170000B76702811387C71F832744FEB307F7001B
:1017100023800700B7970281130710002382E72C6C
:1017200013056004EFF0DFEFB79702812382072CE7
:10173000832744FE938717002322F4FE032744FEE9
:10174000832784FDE34EF7FA834734FEE39C07F4D6
:101750006F00400213000000B797028183C7472C37
:1017600093C7170093F7F70FE39807FE130540069A
:10177000EFF01FEB130000008320C102032481025D
:101780001301010367800000130101FF232681007C
:1017900013040101930700001308000013850700DC
:1017A000930508000324C1001301010167800000B4
:1017B000130101FE232E810013040102232604FEDF
:1017C0006F008004B76702810327C4FE1317270048
:1017D0009387C721B307F7001307300023A0E70062
:1017E000B77702810327C4FE131727009387C72109
:1017F000B307F7001307200023A0E7008327C4FEE8
:10180000938717002326F4FE0327C4FE9307F00FE7
:10181000E3DAE7FA130000000324C1011301010217
:1018200067800000130101FD232611022324810299
:1018300013040103232EA4FCB7070081138587112D
:10184000EFE0DFF8232604FE6F0080058327C4FE47
:10185000638E07008327C4FE93F7F70063980700A1
:10186000B70700811385C713EFE05FF68327C4FE37
:10187000939727000327C4FDB307F70083A707004A
:1018800013850700EFE05FF8B707008113850714A1
:10189000EFE0DFF38327C4FE938717002326F4FECF
:1018A0000327C4FE9307F00FE3D2E7FAB7070081DE
:1018B00013854714EFE09FF1130000008320C1025D
:1018C000032481021301010367800000130101FF5B
:1018D000232611002324810013040101EFF05FEDA2
:1018E000B76702811385C721EFF0DFF3930700008C
:1018F000138507008320C100032481001301010127
:0419000067800000FC
:02000004810079
:10000000300000003100000032000000330000002A
:10001000340000003500000036000000370000000A
:10002000380000003900000061000000620000009C
:10003000630000006400000065000000660000002E
:100040007761697420666F723A200000466F756EA2
:10005000643A20003000000031000000320000004F
:1000600033000000340000003500000036000000BE
:100070003700000038000000390000006100000077
:1000800062000000630000006400000065000000E2
:10009000660000000A00000030000000310000008F
:1000A0003200000033000000340000003500000082
:1000B0003600000037000000380000003900000062
:1000C00061000000620000006300000064000000A6
:1000D00065000000660000003000000031000000F4
:1000E0003200000033000000340000003500000042
:1000F0003600000037000000380000003900000022
:100100006100000062000000630000006400000065
:1001100065000000660000002D2D2D2D2D2D2D2DAC
:100120002D2D2D2D2D2D2D2D2D2D2D2D2D2D2D2DFF
:100130002D2D2D2D2D2D2D0A000000000A00000070
:10014000200000000A2D2D2D2D2D2D2D2D2D2D2D96
:100150002D2D2D2D2D2D2D2D2D2D2D2D2D2D2D2DCF
:060160002D2D2D2D0A00DB
:100168000000008104000081080000810C0000816B
:100178001000008114000081180000811C0000811B
:100188002000008124000081280000812C000081CB
:100198003000008134000081380000813C0000817B
:1001A80054000081580000815C00008160000081DB
:1001B80064000081680000816C000081700000818B
:1001C80074000081780000817C000081800000813B
:1001D80084000081880000818C00008190000081EB
:1001E800980000819C000081A0000081A40000818B
:1001F800A8000081AC000081B0000081B40000813B
:10020800B8000081BC000081C0000081C4000081EA
:10021800C8000081CC000081D0000081D40000819A
:10022800D8000081DC000081E0000081E40000814A
:10023800E8000081EC000081F0000081F4000081FA
:10024800F8000081FC0000810001008104010081A8
:10025800080100810C010081100100811401008156
:040000058000000077
:00000001FF
